:10000000E8289200280884000930930003100D208E
:10001000920C930B072803140D288413A51D1C288C
:1000200000082604251D26068000841700082604E3
:10003000031C26068000272800082604031C260629
:100040002519260680008417260980052728250DF6
:1000500006398C0030208D008C0A302000004A28A0
:1000600000308A000C0882070134753403341534DB
:1000700000343C340C34D9348F018E00FF308E07AD
:10008000031C8F07031CE32803308D00DF304A2058
:100090003E288D01E83E8C008D09FC30031C53285E
:1000A0008C07031850288C0764008D0F50280C18FB
:1000B00059288C1C5D2800005D28080093019200DF
:1000C0001C308E006F308F00CD200F3083168104DE
:1000D0008312FF3063008C07031C8D0703186A2806
:1000E000E3288C001130FF3E8C0D8D0D031C73280E
:1000F000E32803108C0D8D0DFF3E031879280C08A2
:10010000E32803108D0C8C0CFF3E031881280C088B
:10011000E3288D018F018E0002309A288E00013075
:100120009A288D018F018E0004309A288D018F014D
:100130008E00053094000F080D02031DA1280E0843
:100140000C02043003180130031902301405031D9A
:10015000FF30E3280038031DFF300405031DFF3086
:10016000E32891019001103092000D0D900D910D3A
:100170000E0890020F08031C0F0F91020318C728E6
:100180000E0890070F0803180F0F910703108C0D2E
:100190008D0D920BB5280C08E328103094008D01CA
:1001A0008C01930C920C031CDB280E088C070F08A3
:1001B00003180F0F8D078D0C8C0C910C900C940B69
:1001C000D1281008E3288313031383126400080066
:1001D00083168510FF3086008312861483168610DE
:1001E00083120514831605108312AA01AB01C910EE
:1001F0004911C9114914C8010F30CB000F30CA0092
:100200006400851D0A2949147830AC006930AD00BE
:10021000FA21102949102830AC002330AD00F42118
:1002200048088C008D0104307C209E000D089F0042
:100230004A081E07CB0006108316061041308312B1
:100240003C2006148316061006308312A8000230E4
:10025000A6000230A5004B080120F030012006085E
:100260008C008D0102308420CB0064004B083F3CA1
:10027000031D48292A088C002B088D002D088F00AB
:100280002C088E20031D1F2AAA0A0319AB0A4A292B
:10029000AA01AB014B088C008D0102308420CA00FA
:1002A0006400CB1CD2290030491901308C00013088
:1002B00089209E000030C91901308C00003089204F
:1002C000A0001E0884002008AA20A000A100480861
:1002D0008C0004309120A200200821048400220810
:1002E000AA20A200A3006400220823040319942971
:1002F000013048079E009F019F0D1E088C001F08BB
:100300008D0004308E008F01B1201008C800CA0192
:1003100064004A084802031C9229102264303C20E1
:10032000CA0F88290F30CA004911C91164004B1C3B
:10033000A92964004808053C031DA0290330C80012
:10034000C91064004808043C031DA8294C08C800D3
:10035000102948088C00033096209E0048088C0025
:1003600005309620A0001E0884002008AA20031D46
:10037000BC290530C800102964004808043C031952
:10038000C5294808CC000430C8006400C918D12928
:1003900064004A080F3C031DCF29C914D1290F302E
:1003A000CA00102964004919DE2964004A080F3C7C
:1003B0000319DD290F30CA001029491564004A08C5
:1003C0000F3C03191029C9150F304A069E00003052
:1003D0009F001F088D001E0871209E009F011E03B4
:1003E000C8000F30CA001029012232303C200122FF
:1003F00032303C20012232303C20012232303C207D
:100400000800CB01640033304B0203180F2A851417
:1004100001303C20851001303C20CB0F022A08001F
:10042000CB0164000B304B0203181E2A85140130E7
:100430003C20851001303C20CB0F112A0800831688
:10044000851064008312491C272AFA21282AF421E6
:100450008316FF308500FF3086001E3083125E2039
:020460001F2A51
:02400E00F53F7C
:00000001FF
